:10000000830100308A003328A00003088301D30055
:1000100083120C1C2D28FF308F00D0308E00A50FCE
:100020001D28A408031915280511A308031D05128E
:10003000A108031929288512292825082402031C50
:10004000051525082302031C051625082102031C9B
:1000500085162208031DA2030C1083125308830087
:10006000A00E200E09002130840048304520830175
:100070000330D200FD30D100483084004A3049209E
:100080008301C92904068001840A0406031D42284D
:100090000034CA0054208000840A04084A06031968
:1000A00000344A288312D100D21B5D2852088A00EE
:1000B0005108D10A0319D20A8200831352188317F8
:0A00C0005108D10A8400000808006E
:10023A008312AC00A4002A08A3002B08A10008001E
:10024A008312BE01BF010C30A2002208031D2A2915
:10025A00BE0A0319BF0A00303F02503003193E029A
:10026A000318080028298312BF1B40293F08CB0026
:10027A003E08CA004A2983123F08CB003E08CA003A
:10028A00CA09CB09CA0A0319CB0A83120800CE018C
:10029A00CF010310CD0CCC0C031C5A294A08CE07F7
:1002AA004B0803184B0ACF070310CA0DCB0D4C0895
:1002BA004D04031900344E298312C1004008CD00B1
:1002CA003F08CC004108CA00CB013E08CA02031C01
:1002DA00CB03AE234E08C2004F08C300CB0042082E
:1002EA00CA0008008B130B1383120511051285121D
:1002FA000B3083168500D0308100FF3083128F00C7
:10030A00D0308E000C1083160C14831210140B17A5
:10031A008B1708008312AA00AB01AC01992983123A
:10032A002521AB0A0319AC0A1430CC00CD012A08E6
:10033A00CA00CB014C214F082C02031DA6294E08E6
:10034A002B020318080094298312C3004208CD0027
:10035A004108CC004008CB003F08CA004C213E08A7
:10036A00CE070318CF0A4E08C6004F08C700460832
:10037A004302C4004708031C470AC501C5024508D1
:10038A00CB004408CA000800831277215122EC21CD
:10039A00A800EC21A700EC21A900EC21A60004305A
:1003AA0029020318DA290430A9001A302902031C89
:1003BA00E0291930A9002708AA002608AB00290855
:1003CA00AC00AD012808992214308F21CC290A30BB
:1003DA00CA0083124908CD004808CC00CC01043079
:1003EA00CD05CA0AFB290310CD0CCC0CCA0BF8297F
:0603FA004908CB00480891
:10040000CA00CA010230CB050930CE000310CB0C64
:10041000CA0CCE0B062A4C084A06AA004D084B0609
:10042000AB000310C80DC90D2A08C8042B08C90465
:100430004808080083123E0884003F088007C2086D
:1004400003190800410884000008CA00840A000853
:10045000CB004A0403190800410884000008CA00C0
:10046000840A0008CB00803ACC0080304C02013076
:1004700003194A023E088400031C482A800A4108E6
:10048000840001308002840A031C80038403080076
:1004900080034108840001308007840A0318800A21
:1004A0000800FF308312AA00AB000230AC00AD019F
:1004B000FF308312992201308F21AA01AB01023053
:1004C000AC00AD010030992201308F21AA01AB01AF
:1004D000FF301D2101308F21FF30AA00AB011D210B
:1004E00001308F21FF30AA00AB0100301D21013007
:1004F0008F21FF30AA00AB0000301D2101308F2179
:10050000FF30AA00AB001D2101308F21AA01FF306E
:10051000AB001D2101308F21AA01FF30AB0000305C
:100520001D2101308F21AA01AB0100301D210130B6
:100530008F298312B1001430CC00CD012C08CA00E1
:100540002D08CB004C214E08AC004F08AD0024080C
:10055000BE002C08BF002D08C000310883126121A5
:100560004A08B6004B08B7002308BE002C08BF009D
:100570002D08C0002A0861214A08B4004B08B500C4
:100580002108BE002C08BF002D08C0002B086121E7
:100590004A08B2004B08B3002408BE003608BF006A
:1005A0003708C0002C08C1002D08C2003108A9215D
:1005B0004A08BC004B08BD002308BE003408BF0039
:1005C0003508C0002C08C1002D08C2002A08A92146
:1005D0004A08BA004B08BB002108BE003208BF0021
:1005E0003308C0002C08C1002D08C2002B08A92127
:1005F0004A08B8004B08B9003D083C040319112B08
:100600003C08BE003D08BF0038214B08CD004A0819
:10061000CC002D08CB002C08CA00C3234E08B00024
:10062000122BB0013B083A040319272B3A08BE00ED
:100630003B08BF0038214B08CD004A08CC002D08EC
:10064000CB002C08CA00C3234E08AF00282BAF01F3
:100650003908380403193D2B3808BE003908BF009B
:1006600038214B08CD004A08CC002D08CB002C08BF
:10067000CA00C3234E08AE003E2BAE012430BE009C
:100680003608BF003708C0003C30C100B008031D69
:100690004B2BCA015A2B83123008CC00CD012D08F8
:1006A000CB002C08CA00C3234B084A0400300319AE
:1006B0000130CA00CB014A088312C20031081A2255
:1006C0002330BE003408BF003508C0003A30C100F6
:1006D000AF08031D6D2BCA017C2B83122F08CC00A1
:1006E000CD012D08CB002C08CA00C3234B084A04B7
:1006F000003003190130CA00CB014A088312C2003E
:100700002A081A222130BE003208BF003308C00078
:100710003830C100AE08031D8F2BCA019E2B8312F7
:100720002E08CC00CD012D08CB002C08CA00C32315
:100730004B084A04003003190130CA00CB014A08B3
:100740008312C2002B081A222521AC080319AD031D
:10075000AC032D082C04031908003E2BD001CB1F3D
:10076000B82BCA09CA0A0319CB03CB095017D017F3
:100770004D088039D006CD1FC42BCC09CC0A0319F3
:10078000CD03CD09C42BD001CE01CF014C084D04BF
:10079000031DCD2BCA01CB0100341F30D004031040
:1007A000D00ACC0DCD0D031CD02BCD0CCC0C4D089C
:1007B0004B02031DDD2B4C084A02031CE52B4C08A1
:1007C000CA024D08031C4D0ACB02CE0DCF0DD00B33
:1007D000D01AD52BD01FF12BCE09CE0A0319CF0387
:1007E000CF094E08CC004F08CD00501F0034CA0975
:0E07F000CA0A0319CB03CB0900340034953438
:02400E00C43FAD
:00000001FF
